:020000040000FA
:020000000428D2
:08000800FF30A100FF30A2004F
:10001000FF30A300FF30A4000F30A5008A110A12A0
:100020007C20A7178A110A128420A4138A110A12AD
:100030009C20A6118A110A128A20A3118A110A1281
:10004000A220A6128A110A128720A3128A110A126C
:100050009F2026148A110A129320A6148A110A12CC
:10006000902026158A110A128D2023108A110A1257
:10007000AB20A3108A110A12A82023118A110A1298
:10008000A520A8010130A9008A110A12B920403028
:1000900094008A110A12BC20203094002908A80775
:1000A0002808FF3C8A110A12031D5B28FF30A900B3
:1000B0008A110A126228A8088A110A12031D6228EE
:1000C0000130A900A7138A110A128420233093005B
:1000D0000000000000000000000000000000000020
:1000E00028089300A7178A110A1284208A110A127D
:1000F00044288A110A1279288A110A12B920073075
:100100009F008A110A12BC288A110A1296288A11A5
:100110000A1299288A110A1299288A110A12992812
:100120008A110A1299288A110A1299282708880028
:1001300008002608870008008A110A12AE288A11D2
:100140000A12B6288A110A12B6288A110A12B6288B
:100150008A110A12B6288A110A12B62824088A11AE
:100160000A12B92088008A110A12BC2823086700E5
:0E01700008008316031308008312031308000F
:02400E00723FFF
:00000001FF
